:100000000C94E7030C940F040C940F040C940F044D
:100010000C940F040C940F040C940F040C940F0414
:100020000C940F040C940F040C940F040C940F0404
:100030000C940F040C940F040C940F040C940F04F4
:100040000C9476110C940F040C940F040C940F0470
:100050000C940F040C940F040C940F040C940F04D4
:100060000C94C0110C940F0489088C088F08920816
:10007000950898089B089E08A108A408A708E916F7
:10008000D516C116AD169916851671165D1665162C
:1000900078168B169E16B116C416D716EA16491690
:1000A000351621160D16FD161117251739176C1662
:1000B00080169416A816BC16D016E416F8161A1652
:1000C0003F1664168916AE16D316F8161D17F214CD
:1000D00017153C1561158615AB15D015F515282992
:1000E0002A2B2C2D2E2F1320121121100722081835
:1000F00006091905230A1A040B1B03240C1C020D04
:100100001D25010E1E000F1F26141527161720008F
:100110002020002000200020204368616E6E656C66
:10012000202020205253534900204D487A002E00B1
:100130004F4646004F4E200020004578697420202D
:10014000202020202020202020200052657365746C
:100150002053657474696E6773202000546573744E
:1001600020416C61726D20202020202000446973A2
:10017000706C6179204C6F772042616E640053632C
:100180007265656E205361766572202020200053D1
:10019000686F7720537461727473637265656E0063
:1001A000426174746572792043616C69622E20200B
:1001B00000416C61726D204C6576656C20202020BA
:1001C00020004261747465727920416C61726D2007
:1001D0002020004C69506F203373204D6574657288
:1001E000202020004C69506F203273204D657465CB
:1001F0007220202000466C69702053637265656E22
:1002000020202020200000000000240027002A00D9
:1002100000000000250028002B00323031372D303F
:10022000332D31300076312E352062792044766FBF
:10023000676F6E656E004359434C4F502B00352E4F
:1002400036352020202020352E3820202020203533
:100250002E393500352E33352020202020352E36FE
:100260002020202020352E39350020204368616E63
:100270006E656C202020205253534900204D487A4F
:10028000005343414E0000000000003E5B4F5B3EC8
:100290003E6B4F6B3E1C3E7C3E1C183C7E3C181C4B
:1002A000577D571C1C5E7F5E1C00183C1800FFE742
:1002B000C3E7FF0018241800FFE7DBE7FF30483AE8
:1002C000060E2629792926407F050507407F05254A
:1002D0003F5A3CE73C5A7F3E1C1C08081C1C3E7FD2
:1002E00014227F22145F5F005F5F06097F017F0099
:1002F0006689956A606060606094A2FFA2940804B9
:100300007E040810207E201008082A1C08081C2AD9
:1003100008081E101010100C1E0C1E0C30383E3831
:1003200030060E3E0E06000000000000005F0000D8
:100330000007000700147F147F14242A7F2A122349
:100340001308646236495620500008070300001C59
:100350002241000041221C002A1C7F1C2A08083E62
:100360000808008070300008080808080000606075
:100370000020100804023E5149453E00427F4000E3
:1003800072494949462141494D331814127F1027BB
:10039000454545393C4A494931412111090736490A
:1003A000494936464949291E0000140000004034DE
:1003B00000000008142241141414141400412214E3
:1003C0000802015909063E415D594E7C1211127C0A
:1003D0007F494949363E414141227F4141413E7F6B
:1003E000494949417F090909013E414151737F084B
:1003F00008087F00417F41002040413F017F0814F1
:1004000022417F404040407F021C027F7F04081051
:100410007F3E4141413E7F090909063E4151215E2F
:100420007F09192946264949493203017F01033FC3
:100430004040403F1F2040201F3F4038403F631452
:1004400008146303047804036159494D43007F4154
:1004500041410204081020004141417F0402010291
:1004600004404040404000030708002054547840B6
:100470007F284444383844444428384444287F384A
:100480005454541800087E090218A4A49C787F08CC
:1004900004047800447D40002040403D007F102847
:1004A000440000417F40007C047804787C08040408
:1004B000783844444438FC1824241818242418FCA0
:1004C0007C08040408485454542404043F44243C45
:1004D0004040207C1C2040201C3C4030403C4428B4
:1004E0001028444C9090907C4464544C440008364E
:1004F00041000000770000004136080002010204BC
:10050000023C2623263C1EA1A161123A4040207ADB
:100510003854545559215555794122545478422123
:100520005554784020545579400C1E52721239555A
:100530005555593954545459395554545800004557
:100540007C410002457D420001457C407D12111234
:100550007DF0282528F07C545545002054547C54C7
:100560007C0A097F4932494949323A4444443A3283
:100570004A4848303A4141217A3A42402078009D29
:10058000A0A07D3D4242423D3D4040403D3C24FFD5
:100590002424487E4943662B2FFC2F2BFF0929F684
:1005A00020C0887E090320545479410000447D41D5
:1005B0003048484A32384040227A007A0A0A727D2E
:1005C0000D19317D2629292F282629292926304849
:1005D0004D4020380808080808080808382F10C8B7
:1005E000ACBA2F102834FA00007B000008142A143B
:1005F0002222142A14085500550055AA55AA55AAB6
:10060000FF55FF55FF000000FF00101010FF001401
:100610001414FF001010FF00FF1010F010F014145D
:1006200014FC001414F700FF0000FF00FF1414F482
:1006300004FC141417101F10101F101F1414141F83
:1006400000101010F0000000001F101010101F10FC
:10065000101010F010000000FF10101010101010FB
:100660001010FF10000000FF140000FF00FF00004A
:100670001F10170000FC04F414141710171414F4BE
:1006800004F40000FF00F714141414141414F700F9
:10069000F7141414171410101F101F141414F4144A
:1006A0001010F010F000001F101F0000001F1400B9
:1006B0000000FC140000F010F01010FF10FF1414E4
:1006C00014FF141010101F00000000F010FFFFFFB7
:1006D000FFFFF0F0F0F0F0FFFFFF0000000000FF70
:1006E000FF0F0F0F0F0F3844443844FC4A4A4A3476
:1006F0007E02020606027E027E026355494163388D
:1007000044443C04407E201E2006027E020299A53D
:10071000E7A5991C2A492A1C4C7201724C304A4D9B
:100720004D303048784830BC625A463D3E494949D0
:10073000007E0101017E2A2A2A2A2A44445F444479
:1007400040514A444040444A51400000FF0103E008
:1007500080FF000008086B6B083612362436060F3F
:10076000090F06000018180000001010003040FFAC
:100770000101001F01011E00191D1712003C3C3C25
:100780003C000000000000000000230026002900BB
:100790000404040404040404020202020202030327
:1007A000030303030102040810204080010204082F
:1007B00010200102040810200000000800020100BF
:1007C0000003040700000000000000001A1C1124B0
:1007D0001FBECFEFD8E0DEBFCDBF24E0A4E8B3E07A
:1007E00001C01D92A538B207E1F713E0A0E0B1E027
:1007F000E0EEFDE302C005900D92A438B107D9F7F1
:1008000013E0C7EED3E004C02197FE010E946B1CE9
:10081000C63ED107C9F70E949E150C94EE1E0C949B
:1008200000000F931F93CF93DF93DC0155968C91BB
:100830005597823071F0833009F1813009F08CC016
:100840001496ED91FC911597E41BF50BE21BF30B4D
:1008500020C01496ED91FC911597CF01861B970B44
:10086000BC01615071091696ED91FC911797CF016B
:10087000841B950BAC01421B530B6EC01696ED9179
:10088000FC911797CF01861B970BBC016150710932
:10089000FA0177FD1BC116968D919C9117976817E9
:1008A00079070CF013C1F7FF04C02E0F3F1FE0E0E3
:1008B000F0E014968D919C911597AF01420F531F54
:1008C000841795071CF49C012E1B3F0B1216130670
:1008D0000CF0FCC0CB0177FD079643E0959587951A
:1008E0004A95E1F79695982F882797958795E80F71
:1008F000F91FEE5FFE4F6770772781E090E001C03F
:10090000880F6A95EAF7482F0130110541F088F009
:100910000230110509F0DAC02E0F3F1F15C02E0F4F
:100920003F1FE217F30709F4D1C08081842B819324
:10093000F8CF80952E0F3F1FE217F30709F4C6C0CA
:10094000908198239193F8CFE217F30709F4BEC082
:10095000808184278193F8CF77FDB8C014968D915C
:100960009C911597681779070CF0B0C057FF04C029
:10097000240F351F40E050E016968D919C911797FB
:10098000FA01E20FF31F8E179F071CF49C01241B32
:10099000350B121613060CF099C0A22F842F8695E2
:1009A0008695869590E8899F600D711D1124FB0145
:1009B000EE5FFE4F4770A9F198E0941B492F50E07D
:1009C000EA01C25FDC4F8881291790F4421B51096C
:1009D0002FEF30E002C0359527954A95E2F7822344
:1009E0000130110541F068F00230110589F06EC048
:1009F0000130110519F42081822B0CC00130110542
:100A000020F480952081822305C00230110531F445
:100A1000208182278083A91708F458C0A91BE058B9
:100A2000FF4FA83048F10230110559F4EF018A2F29
:100A3000988190959883C058DF4F88508830C0F7D0
:100A400030C081E00130110509F080E08195EF01AF
:100A50009A2F8883C058DF4F98509830D0F788EF8E
:100A60008A0F86958695869590E8899FE00DF11D01
:100A70001124E058FF4FA770AA2341F1B0E0AA5F0C
:100A8000BC4F8C910130110529F038F0023011056E
:100A9000D1F01CC09081892B18C08095908189234A
:100AA00014C088EF8A0F86958695869590E8899F71
:100AB000E00DF11D1124E058FF4FA77039F0B0E0B0
:100AC000AA5FBC4F8C91908189278083DF91CF9161
:100AD0001F910F9108950F931F93CF93DF93DC0124
:100AE000FB0155968C915597823081F0833019F136
:100AF000813051F514968D919C911597BC01641B22
:100B0000750BAB0141505109BF0181C014966D9125
:100B10007C911597CB018E1B9F0BFC0116968D9136
:100B20009C911797BC01641B750BAB014150510997
:100B3000E21BF30B09C016966D917C9117976E1B03
:100B40007F0B621B730B63C057FD1CC116968D9102
:100B50009C911797481759070CF014C1F7FF04C070
:100B60002E0F3F1FE0E0F0E014968D919C911597B9
:100B7000BF01620F731F861797071CF49C012E1B81
:100B80003F0B121613060CF0FDC0CA0157FD079665
:100B900063E0959587956A95E1F79695982F882754
:100BA00097958795E80FF91FEE5FFE4F4770552721
:100BB00081E090E001C0880F4A95EAF7482F0130A4
:100BC000110541F088F00230110509F0DBC02E0F4D
:100BD0003F1F15C02E0F3F1FE217F30709F4D2C0C5
:100BE0008081842B8193F8CF80952E0F3F1FE217D1
:100BF000F30709F4C7C0908198239193F8CFE217C7
:100C0000F30709F4BFC0808184278193F8CF57FD93
:100C1000B9C014968D919C911597481759070CF0FF
:100C2000B1C077FF04C0260F371F60E070E0169652
:100C30008D919C911797FB01E20FF31F8E179F0771
:100C40001CF49C01261B370B121613060CF09AC0DD
:100C5000A22F862F86958695869590E8899F400DD0
:100C6000511D1124FA01EE5FFE4F6770A9F198E063
:100C7000961B492F50E0EA01C25FDC4F888129179B
:100C800090F4421B51092FEF30E002C035952795B3
:100C90004A95E2F782230130110541F068F00230F5
:100CA000110589F06FC00130110519F42081822BE4
:100CB0000CC00130110520F480952081822305C0ED
:100CC0000230110531F4208182278083A91708F4AE
:100CD00059C0A91BE058FF4FA83048F10230110558
:100CE00059F4EF018A2F988190959883C058DF4F6F
:100CF00088508830C0F731C081E00130110509F01B
:100D000080E08195EF019A2F8883C058DF4F98507B
:100D10009830D0F788EF8A0F86958695869560E89B
:100D2000869FE00DF11D1124E058FF4FA770AA2304
:100D300049F1B0E0AA5FBC4F8C910130110529F058
:100D400038F002301105D9F01DC09081892B03C005
:100D5000809590818923808315C088EF8A0F8695BE
:100D60008695869570E8879FE00DF11D1124E05867
:100D7000FF4FA77039F0B0E0AA5FBC4F8C91908113
:100D80008927E9CFDF91CF911F910F910895FC0141
:100D900077FD9AC080859185681779070CF094C01B
:100DA00057FD92C082859385481759070CF08CC077
:100DB0008589823009F07CC084819581DC01A61B85
:100DC000B70BBD016150710986819781FC01E41B5D
:100DD000F50BAF01415051090AC0813041F48481C3
:100DE0009581841B950BAB01BC01615071092130C9
:100DF000310529F008F122303105E1F10895FA01B9
:100E000057FD3796A3E0F595E795AA95E1F7F69596
:100E1000FE2FEE27F795E7956E0F7F1FFB01EE5F24
:100E2000FE4F4770552781E090E001C0880F4A953A
:100E3000EAF79081892B3AC0FA0157FD379623E0F3
:100E4000F595E7952A95E1F7F695FE2FEE27F795AC
:100E5000E7956E0F7F1FFB01EE5FFE4F4770552732
:100E600081E090E001C0880F4A95EAF78095908173
:100E700089231CC0FA0157FD379683E0F595E79565
:100E80008A95E1F7F695FE2FEE27F795E7956E0F19
:100E90007F1FFB01EE5FFE4F4770552781E090E01A
:100EA00001C0880F4A95EAF79081892780830895C9
:100EB000833009F092CF86819781861B970BBA0108
:100EC000AC014150510993CF089560E082E00E9447
:100ED000C41060E084E00E94C41061E082E00E94DF
:100EE000C41060E082E00C94C41060E082E00E94D4
:100EF000C41061E084E00E94C41061E082E00E94BE
:100F0000C41060E082E00C94C4100F931F93CF9341
:100F1000DF93C62FDEE0D80F8091840326E330E014
:100F2000281B310990910001692F70E000E010E06A
:100F300040E050E086E594E00E9411046D2F70E0DF
:100F400001E010E026E330E040E050E086E594E088
:100F50000E941104D0930001C63320F085E38093F2
:100F6000840302C0C0938403DF91CF911F910F913E
:100F70000C94D5131F93CF93DF938F5D91409C0109
:100F8000369527952F71EC0156E0D695C7955A9561
:100F9000E1F7D695DC2FCC27D795C795C22B61E01A
:100FA00083E00E94C41060E083E00E94C4100E94AD
:100FB00075070E9465070E9465070E9465070E94E9
:100FC000750710E1C0FF03C00E94750702C00E94B0
:100FD0006507D695C7951150A9F70E9465070E942D
:100FE00065070E9465070E94650761E083E00E9433
:100FF000C41060E083E00E94C41060E082E00E94C0
:10100000C41060E084E0DF91CF911F910C94C41074
:1010100092EF980F8E3008F0892F8770982F906488
:1010200080E240E050E090937C0020917A002064C0
:1010300020937A0020917A0026FDFCCF2091780041
:101040006091790030E0362B420F531F815059F7E1
:10105000CA0125E0969587952A95E1F708958FE0D6
:101060000E9408082091900330E02A573140820FF7
:10107000931F65E070E00E94571CCB01C296089553
:10108000CF92DF92EF92FF920F931F93CF93DF9354
:10109000D82FC62E0E94811310926304109262040E
:1010A000109265041092640481E080936A04DD2349
:1010B00019F0CFEFCD0F01C0CBE087E0D82E01E0D3
:1010C00010E09AE0E92EF12CCC3008F0C0E010934B
:1010D0006704009366041092690410926804CD13AB
:1010E0000AC0C11008C010926704109266041093E1
:1010F0006904009368044C2F50E0FA013197EB30FB
:10110000F10520F4EC5CFF4F0C946B1C85EF91E033
:1011100020C084EE91E01DC083ED91E01AC082EC06
:1011200091E017C081EB91E014C080EA91E011C01A
:101130008FE891E00EC08EE791E00BC08DE691E064
:1011400008C08CE591E005C08BE491E002C08AE321
:1011500091E00E947D15109367040093660410923D
:10116000690410926804CD130AC0CC2041F010929B
:10117000670410926604109369040093680488E37E
:1011800091E00E947D15C43020F08AEF8C0F8330EF
:1011900078F4EC2FF0E0E557FC4F8081882319F0BC
:1011A00084E391E002C080E391E00E947D1526C0B7
:1011B000C43021F460918F0370E016C0C530D1F4C3
:1011C0000E942F08B7010E94571C80E090E04AE07F
:1011D0000E943C158EE291E00E947D150E942F082E
:1011E000B7010E94571CBC0180E090E04AE00E94D9
:1011F0003C1504C08EE393E00E942A1583E493E03B
:101200000E942A15CF5FDA94D1105ECFDF91CF9183
:101210001F910F91FF90EF90DF90CF900C94D5131A
:10122000CF92DF92EF92FF920F931F93CF93DF93B2
:1012300090918D0380918C03911103C0882309F450
:10124000E6C0882329F0C4E5D0E004E410E004C03F
:10125000CEE7D0E006E610E00E942F088C179D072D
:1012600008F04AC00817190718F5BC01601B710B7C
:1012700080E090E00E94121D6B017C01CE01801B7A
:10128000910BBC0180E090E00E94121D9B01AC011B
:10129000C701B6010E94711C20E030E048EC52E426
:1012A0000E94A01D0E94E31CC62F653010F00AC0EA
:1012B000C0E082E390E090938A038093890388ECF6
:1012C00090E00AC06F3068F484E690E090938A035F
:1012D0008093890388EE93E090938803809387033B
:1012E00014C0693150F488EC90E090938A038093A5
:1012F000890388EB9BE0F0CFC3E610928A0310923B
:1013000089031092880310928703EE24E394F12C52
:1013100002E010E024E030E040E250E06DE370E0F5
:1013200086E594E00E94A00F04E110E02AE030E09E
:1013300042E250E06AE370E086E594E00E94A00F8C
:10134000E12CF12C00E110E026E030E044E250E036
:101350006CE370E086E594E00E94A00FC63580F053
:10136000EE24E394F12C02E010E024E030E045E2CA
:1013700050E06DE370E086E594E00E94A00F02C0AB
:10138000C23480F0EE24E394F12C02E010E024E07B
:1013900030E048E250E06DE370E086E594E00E94C2
:1013A000A00F02C0CE3280F0EE24E394F12C02E0D4
:1013B00010E024E030E04BE250E06DE370E086E5C1
:1013C00094E00E94A00F02C0CA3180F0EE24E394A2
:1013D000F12C02E010E024E030E04EE250E06DE35A
:1013E00070E086E594E00E94A00F02C0C63078F05D
:1013F000EE24E394F12C02E010E024E030E041E33D
:1014000050E06DE370E086E594E00E94A00FDF916C
:10141000CF911F910F91FF90EF90DF90CF900895A3
:101420000F931F93CF93DF936091940380E090E03C
:101430000E947D1E0BE813E0C0E0D0E0F80161914E
:101440008F012196CE010E947D1EC930D105B1F7D2
:101450006FEE8AE090E0DF91CF911F910F910C9495
:101460007D1EEBE8F3E081E0808311828283838339
:1014700095E0948390E8958386831782808708950A
:10148000E82FF0E0E252FF4FE491F0E0EE0FFF1F93
:10149000E258FF4F859194910895AF92BF92CF92F9
:1014A000DF92EF92FF920F931F93CF93DF93CDB70D
:1014B000DEB766970FB6F894DEBF0FBECDBFB82E6D
:1014C0006B010E94811381E090E090936904809306
:1014D000680490936704809366048AE090E0909398
:1014E000630480936204109265041092640483E0A4
:1014F00080936A048B2D0E94400ABC0180E090E03A
:101500004AE00E943C158BE490E090936304809342
:10151000620487E090E0909365048093640432E075
:10152000A32EA0926A0489E291E00E947D15EE2428
:10153000E394F12C08E110E02FE730E048E150E0BF
:1015400060E070E086E594E00E94EF0F1092630483
:10155000109262048BE190E09093650480936404A0
:1015600081E080936A0487E191E00E947D151092EA
:1015700063041092620487E290E090936504809384
:101580006404A0926A0485E191E00E947D1583E1E4
:1015900091E00E947D150B2D10E002521F4FF801C3
:1015A0008491883010F491E411C0803110F492E4F9
:1015B0000DC0883110F495E409C0803210F496E42F
:1015C00005C0883210F492E501C09CE499838770CD
:1015D0008F5C8A831B82CE0101967C010E942A15B2
:1015E00080E191E00E947D15B60180E090E04AE044
:1015F0000E943C15109263041092620489E390E00B
:10160000909365048093640481E080936A04F801F8
:101610000491083018F466E473E016C0003118F441
:101620006FE473E011C0083118F468E573E00CC092
:10163000003218F465E673E007C0083218F46FE66C
:1016400073E002C069E773E0C7010E94121EF70150
:1016500001900020E9F73197EE19FF09FF27D70124
:10166000AE0FBF1F07700F5C0C93EC0FFD1F1282B3
:10167000F70101900020E9F7C7018E1B9F0B4696EA
:1016800096958795182F112331F08EE091E00E94F6
:101690007D151150F8CFC7010E942A150E9410092C
:1016A0000E94D51366960FB6F894DEBF0FBECDBF6D
:1016B000DF91CF911F910F91FF90EF90DF90CF902E
:1016C000BF90AF900895EF92FF920F931F93CF9327
:1016D000DF938C0180919303882311F0D0E001C047
:1016E000D8E0CD2F8CE2E82EFF24F3948C2F0E94BB
:1016F000400A801B910B1816190634F48C2F0E9497
:10170000400A801B910B07C08C2F0E94400A980151
:10171000281B390BC9018E159F0514F4DC2F7C01A1
:10172000CF5FC03319F78D2FDF91CF911F910F91AC
:10173000FF90EF900895CF92DF92EF92FF920F9378
:101740001F93CF93DF936C017A018B01C0E0D0E04F
:10175000CE15DF0589F0D8016D918D01D601ED918F
:10176000FC910190F081E02DC6010995892B11F4BF
:101770007E0102C02196ECCFC701DF91CF911F916E
:101780000F91FF90EF90DF90CF9008953FB7F894BE
:101790008091FB039091FC03A091FD03B091FE03A7
:1017A00026B5A89B05C02F3F19F00196A11DB11DBC
:1017B0003FBFBA2FA92F982F8827820F911DA11DF7
:1017C000B11DBC01CD0143E0660F771F881F991F33
:1017D0004A95D1F7089585ED8093BC008091BC00B7
:1017E00084FDFCCF1092260408954091D103262F4A
:1017F00030E0240F311D21323105DCF42091260424
:101800002430C9F4FC0180E090E0861758F4309150
:10181000D1032191DC01A155BC4FA30FB11D2C9325
:101820000196F3CF8091D103680F6093D10380E0DC
:10183000089581E0089582E00895089581E090E0A0
:101840003091860320918503321710F480E090E0F8
:1018500091958195910908958091860390918503D2
:10186000891730F48F5F8093860380E090E00895BD
:101870008FEF9FEF08958091850390E0209186037C
:10188000821B91090895CF92DF92EF92FF920F93FE
:101890001F93CF93DF937C01262F972F8A0180918E
:1018A0002704882391F0C62FD72F6E01C40ED51EB2
:1018B000CC15DD0571F06991D701ED91FC91019096
:1018C000F081E02DC7010995F3CF642F822F0E948C
:1018D000F50BC801DF91CF911F910F91FF90EF9011
:1018E000DF90CF900895CF93DF931F92CDB7DEB7EF
:1018F0006983209127042223D1F0209149042032CA
:1019000040F021E030E0FC013383228380E090E06E
:1019100015C080912804E82FF0E0E75DFB4F998126
:1019200090838F5F809328048093490405C061E011
:10193000CE0101960E94F50B81E090E00F90DF91BF
:10194000CF91089508952F923F924F925F926F9298
:101950007F928F929F92AF92BF92CF92DF92EF923F
:10196000FF920F931F93CF93DF93CDB7DEB76B97A3
:101970000FB6F894DEBF0FBECDBF4C015A8349832A
:101980001F830E83FD82EC82CB82DC0158964D9141
:101990005C9159974115510509F0A5C018968D9194
:1019A0009C911997681779070CF05AC11A968D9176
:1019B0009C911B97E981FA81E817F9070CF050C157
:1019C000D12CCB013B81F6E03F9F800D911D11246E
:1019D000181619060CF044C1C60133E0880F991F90
:1019E0003A95E1F749815A81840F951F1816190617
:1019F0000CF036C157968C91811103C0203B08F042
:101A00002F5F55E0259F900111247E876D875B0134
:101A1000212CC901861B970B99878887A981BA81D8
:101A20001896BB87AA87B5E02B1641F0E885F985A3
:101A3000EA0DFB1DEA57FD4F349001C0312C69803F
:101A40007A80230130FE12C0D401ED91FC91BB815C
:101A5000B13031F40480F581E02D2E813F8118C032
:101A60000684F785E02DEE80FF801CC0EC81FD81AF
:101A70002E813F81E217F307E1F0D401ED91FC9153
:101A8000BB81B13051F40480F581E02D2C813D8182
:101A9000A301B501C40109950CC00684F785E02DAA
:101AA000EC80FD8086019601A2016D857E85C401D2
:101AB00009953694EFEF6E1A7E0A4C0C5D1C2A8550
:101AC0003B856216730609F0BDCF23943FEFA31A3E
:101AD000B30A4D855E854C0D5D1D5E874D8756E0D2
:101AE0002512A1CFBDC0FA01349634913297859169
:101AF0009491231BA7E02A9F800D911D1124FA01C8
:101B0000259134913A8B298BFC0125903490FC016E
:101B1000329634913887319644914C873196E491CE
:101B2000FC013596A491319684915B81523050F03E
:101B30006A2E0A2E000C7708E82F082E000CFF0BE7
:101B4000FB87EA87FB81CF2ED12C6C9C90016D9C8A
:101B5000300D7C9C300D1124A901460F571F588B66
:101B60004F871C82A12CEA2FAA0FFF0B3B016E0EA0
:101B70007F1E5885650F711DDB01AE0FBF1FBF8B28
:101B8000AE8BE981FA81E80FF11D87FDFA95F98F97
:101B9000E88F9C85A91608F063C08A2D90E04A85DD
:101BA0005B85480F591F4C9D90014D9D300D5C9DEC
:101BB000300D1124A981BA81A20FB31FBE87AD8752
:101BC0007B8E6A8E4F845888BC81B619BB8BE88D9A
:101BD000F98DE80FF91FFD8BEC8B8B89FA8D8F0F38
:101BE0002A8D3B8D4E895F892417350799F18770BF
:101BF00041F4C1010196E989FA89E20DF31DB4901F
:101C00001C01B7FE1EC0D401ED91FC91BB81B13027
:101C100061F40480F581E02D2E813F814C895D893E
:101C20006A8D7B8DC40109950CC00684F785E02D73
:101C3000EE80FF80860196014D855E85B201C4016C
:101C40000995BB0CEA8DFB8D3196FB8FEA8F4C0C0E
:101C50005D1CC3CF5C818885580F5C83A39499CFAA
:101C60006B960FB6F894DEBF0FBECDBFDF91CF915C
:101C70001F910F91FF90EF90DF90CF90BF90AF90AA
:101C80009F908F907F906F905F904F903F902F909C
:101C90000895AF92BF92CF92EF92FF920F931F934E
:101CA000CF93DF93EC01262F888D998D009709F053
:101CB00042C06A3069F42C898E859F8538E0239F65
:101CC000800D911D11249F878E871D861C86ACC0B8
:101CD0006D3009F4A9C08E898823C1F03C898C85B8
:101CE0009D8546E0349F800D911D112448855985BE
:101CF000841795075CF01D861C868E859F85E8E01D
:101D00003E9F800D911D11249F878E87EA88FB8856
:101D1000088919894E855F856C857D85CC88CE01C3
:101D20000E94A30C2C898C859D85F6E02F9F800D49
:101D3000911D112441C06A3079F41D861C862C89BE
:101D4000FC013696E4918E859F852E9F800D911D16
:101D500011249F878E8768C06D3009F465C0AC017F
:101D60004C5F5F4FFA013491631708F45DC0319600
:101D7000E491E61708F458C0FA014491362F341B59
:101D8000FC013296A590B490F7E03F9FA00CB11CE7
:101D90001124F501329634913196E491332311F0F8
:101DA000E1110DC0F5013496E4912C898C859D8557
:101DB000E29F800D911D11249D878C8735C0F50110
:101DC000359644915E89552311F16C89E32FF0E03B
:101DD000E40FF11D47FDFA956E9FD0016F9FB00D86
:101DE00011244C855D854A0F5B1FE885F9854E17E8
:101DF0005F076CF01D861C86FC013696E4918E858B
:101E00009F856E9F800D911D11249F878E87EA8884
:101E1000FB88088919894E855F856C857D85CC880E
:101E2000CE010E94A30CBECF81E090E0DF91CF9164
:101E30001F910F91FF90EF90CF90BF90AF900895BA
:101E4000EF92FF920F931F93DC01ED91FC9111979C
:101E50001A960D911C911B9718962D913C911997EC
:101E60000684F785E02D7B0140E050E060E070E003
:101E700009951F910F91FF90EF9008956F927F92B7
:101E80008F929F92AF92BF92CF92DF92EF92FF928A
:101E90000F931F93CF93DF936C015A014801EB011D
:101EA0003B01620E731EC615D70574F4D601ED9181
:101EB000FC910084F185E02D87019401A501BE010C
:101EC000C60109952196EFCFDF91CF911F910F9118
:101ED000FF90EF90DF90CF90BF90AF909F908F904A
:101EE0007F906F900895EF92FF920F931F93DC0104
:101EF000ED91FC91260F371F215031090680F781A3
:101F0000E02D78018A0109951F910F91FF90EF90C4
:101F10000895EF92FF920F931F937801DC01ED91EA
:101F2000FC91240F351F8901015011090680F781AA
:101F3000E02D9B0109951F910F91FF90EF9008955F
:101F40006F927F928F929F92AF92BF92CF92DF92C9
:101F5000EF92FF920F931F93CF93DF93EC014B010E
:101F60005A0169013801E881F9810284F385E02D85
:101F700087010995E881F981A501460D571D41505A
:101F800051090284F385E02D9601B401CE01099533
:101F9000E881F9810084F185E02D9301A501B40168
:101FA000CE010995E881F981C80CD91CB6016150B0
:101FB00071090084F185E02D9301A501CE010995F9
:101FC000DF91CF911F910F91FF90EF90DF90CF9015
:101FD000BF90AF909F908F907F906F9008952F92B9
:101FE0003F924F925F926F927F928F929F92AF92A9
:101FF000BF92CF92DF92EF92FF920F931F93CF93F6
:10200000DF9300D01F92CDB7DEB74C017B836A838C
:102010006A01590117019801241B350B37FF03C0D2
:10202000319521953109C5014A815B81841B950B4E
:1020300097FF03C091958195910951E059838217CB
:10204000930714F019820BC09A2D8B2D5801092F7C
:10205000182F9A818B81DB82CA82C92ED82E8A8161
:102060009B81A816B9065CF49C2D8D2D6801092F63
:10207000182F9A818B81BB82AA82A92EB82E2501A6
:10208000AA81BB814A1A5B0A38016C187D0877FE69
:1020900003C0719461947108720157FE03C0BFEFD1
:1020A000EB1AFB0AF594E794C016D1061CF00FEF6B
:1020B0001FEF1FC001E010E01CC0D401ED91FC91A6
:1020C000B9810480F581E02D9101BB23C1F04A81E3
:1020D0005B81B601C4010995E618F708F7FE04C054
:1020E000C00ED11EE40CF51CEA81FB813196FB8306
:1020F000EA834A815B81A416B506FCF604C0A601FA
:102100006A817B81E7CF0F900F900F90DF91CF9185
:102110001F910F91FF90EF90DF90CF90BF90AF9005
:102120009F908F907F906F905F904F903F902F90F7
:1021300008950E940D1E833081F028F4813099F0BB
:102140008230A1F008958730A9F08830B9F084304A
:10215000D1F4809180008F7D03C0809180008F77C3
:1021600080938000089584B58F7702C084B58F7DF9
:1021700084BD08958091B0008F7703C08091B00036
:102180008F7D8093B00008951F93CF93DF93282F06
:1021900030E0F901E854F84F8491F901EC55F84F1B
:1021A000D491F901E057F84FC491CC23C9F0162F10
:1021B00081110E949B10EC2FF0E0EE0FFF1FE05FFB
:1021C000FD4FA591B4918FB7F894111105C09C9162
:1021D000ED2FE095E92302C0EC91ED2BEC938FBF3E
:1021E000DF91CF911F910895CF93DF9390E0FC0191
:1021F000EC55F84F2491FC01E057F84F8491882367
:1022000061F190E0880F991FFC01EA5FFD4FC591D5
:10221000D491FC01E05FFD4FA591B491611109C01B
:102220009FB7F8948881209582238883EC912E2390
:102230000BC0623061F49FB7F8943881822F80958B
:1022400083238883EC912E2B2C939FBF06C08FB7DE
:10225000F894E8812E2B28838FBFDF91CF910895CA
:102260008F929F92AF92BF92CF92DF92EF92FF92A6
:102270006B017C010E94C60B4B015C01C114D104AF
:10228000E104F104F1F00E94C60BDC01CB018819D6
:102290009909AA09BB09883E9340A105B10570F3CD
:1022A00021E0C21AD108E108F10888EE880E83E027
:1022B000981EA11CB11CC114D104E104F10419F74A
:1022C000DDCFFF90EF90DF90CF90BF90AF909F90C9
:1022D0008F9008952FB7F8946091F7037091F803E9
:1022E0008091F9039091FA032FBF08951F920F92E6
:1022F0000FB60F9211242F933F938F939F93AF9319
:10230000BF938091F7039091F803A091F903B091E6
:10231000FA033091F60326E0230F2D3720F40296BE
:10232000A11DB11D05C029E8230F0396A11DB11DF4
:102330002093F6038093F7039093F803A093F90397
:10234000B093FA038091FB039091FC03A091FD03ED
:10235000B091FE030196A11DB11D8093FB039093E4
:10236000FC03A093FD03B093FE03BF91AF919F9137
:102370008F913F912F910F900FBE0F901F90189546
:102380001F920F920FB60F9211242F933F934F93EA
:102390005F936F937F938F939F93AF93BF93EF93CD
:1023A000FF938091B900887F803609F49CC068F55E
:1023B000883209F45BC090F4803109F454C038F4D9
:1023C000882309F4F6C0883009F44DC0F6C088317E
:1023D00009F44CC0803209F45DC0EFC0803409F4C8
:1023E00068C048F4803309F455C0883309F0E5C06B
:1023F00080932404D8C0803509F44FC0883509F48F
:102400005DC0883409F0D9C0D6C0883909F4C7C086
:10241000A8F4883709F467C038F4883609F463C033
:10242000803709F460C0C9C0883809F4B8C0803961
:1024300009F45FC0803809F0C0C05BC0803B09F47C
:1024400086C038F4803A09F466C0883A09F47FC03F
:10245000B4C0803C09F4A7C0883C09F4A4C0883B00
:1024600009F48AC0AAC08091010410C0909123048D
:1024700080912204981770F5E091230481E08E0F7B
:1024800080932304F0E0EE5FFB4F80818093BB00DC
:1024900085EC86C0809324048EC0E091230481E003
:1024A0008E0F809323048091BB00F0E0EE5FFB4F22
:1024B000808390912304809122046EC0E0912304D4
:1024C00081E08E0F809323048091BB00F0E0EE5FEB
:1024D000FB4F80838091250481116DC081E0809342
:1024E000000484EA61C083E0809326041092F5031F
:1024F000CFCF8091F503803208F051C0E091F50311
:1025000081E08E0F8093F5038091BB00F0E0EB52E9
:10251000FC4F8083BDCF85EC8093BC0010922604D5
:102520008091F503803230F4E091F503F0E0EB5256
:10253000FC4F10826091F50370E0E091D303F091BD
:10254000D40385ED93E009951092F50336C084E03D
:10255000809326041092D2031092D103E091CF030E
:10256000F091D00309958091D103811105C081E0DC
:102570008093D1031092AF03E091D20381E08E0FDC
:102580008093D203F0E0E155FC4F80818093BB0043
:102590009091D2038091D103981708F479CF85E800
:1025A0008093BC000AC085EC8093BC001092260486
:1025B00004C0109224040E94EB0BFF91EF91BF9195
:1025C000AF919F918F917F916F915F914F913F91CB
:1025D0002F910F900FBE0F901F90189520914904D6
:1025E00090918404213208F04AC080912604811120
:1025F000FCCF32E03093260431E0309325043FEFE6
:10260000309324041092230420932204A9E2B4E01E
:1026100042E054E0FA013E2F341B321718F43D918A
:102620003193F9CF1092010420910104990F922B5C
:102630009093010490910004913061F41092000491
:10264000909101049093BB009091BC0093FDF8CF52
:1026500095EC01C095EE9093BC00909126049230C9
:10266000E1F3909124049F3F79F08091240480321B
:1026700041F080912404803331F084E005C081E092
:1026800003C082E001C083E0109228041092490444
:1026900010922704089590917704992339F08EBD04
:1026A00000000DB407FEFDCF8EB5089528E030E0A0
:1026B00040E8E0917A04F0917B045081909181048C
:1026C000909595239083E0917804F091790490910E
:1026D0008004542F582319F05081952B03C050814A
:1026E000909595239083E0917A04F0917B0450813A
:1026F00090918104952B9083469521503109C9F61C
:10270000089580E092E0E2E0F1E0DF019C011D929B
:1027100021503040E1F70895CF93C82F8091720483
:102720008F3F59F1E0917C04F0917D04808190917C
:102730008204982B9083E0917E04F0917F042081A5
:1027400090918304909592239083E0917C04F09182
:102750007D042081909182049095922390838C2F08
:102760000E944B13E0917C04F0917D049081809154
:102770008204892B8083CF9108958091700491E029
:1027800090932704809384041092280410924904A3
:1027900060E08AE494E00E94730C6C2F8AE494E079
:1027A0000E94730CCF910C94EE12EF92FF920F9354
:1027B0001F93CF93DF9381E20E948C1380E00E94ED
:1027C0008C138FE70E948C1382E20E948C1380E0AE
:1027D0000E948C1383E00E948C13809172048F3FBF
:1027E00079F1E0917C04F0917D04908180918204E4
:1027F000892B8083E0917E04F0917F049081809109
:102800008304892B8083E0917C04F0917D04908186
:1028100080918204809589238083C2E0D1E08991F0
:102820000E944B1383E0C230D807C9F7E0917C04C3
:10283000F0917D04908180918204892B808330C047
:10284000F090B8008CE08093B800C2E0D1E0EE24B4
:10285000E39480917004E0922704809384041092A2
:1028600028041092490460E48AE494E00E94730C06
:1028700000E010E0FE01E00FF11F60818AE494E0C7
:102880000E94730C0F5F1F4F0031110599F70E94D2
:10289000EE12609683E0C230D807D9F6F092B80005
:1028A000DF91CF911F910F91FF90EF900895CF93FB
:1028B000DF93EDEBF7E08491E9EAF7E0D491E5E905
:1028C000F7E0C491CC2391F081110E949B10EC2F72
:1028D000F0E0EE0FFF1FEA57F84FA591B491EC918D
:1028E000ED2381E090E021F480E002C080E090E000
:1028F000DF91CF9108950F931F93CF930E945714A8
:102900000197D1F100E010E00E945714892B49F49F
:102910000F5F1F4F65E070E080E090E00E94301193
:10292000F3CFC801805591098C3D910528F00C32F8
:10293000114020F0C4E003C0C3E001C0C1E08091B9
:10294000FF03811103C000E010E011C01092FF03EB
:10295000C130C9F785E020C00F5F1F4F0932110554
:10296000A1F065E070E080E090E00E9430110E94EC
:102970005714019719F4F0CF80E00EC0083211050A
:1029800021F00E945714892B11F08C2F05C00E9452
:102990005714892BE1F382E0CF911F910F91089595
:1029A000CF93DF93EC0161E086E00E94F410209762
:1029B00011F460E004C0CF3FD10531F461E086E05E
:1029C000DF91CF910C94C410EEEBF7E0E491E3308B
:1029D000F9F048F4E130B9F0E230A1F584B5806255
:1029E00084BDC8BD34C0E730E9F0E83019F1E43007
:1029F00049F580918000806280938000D0938B00A5
:102A0000C0938A0024C084B5806884BDC7BD1FC040
:102A100080918000806880938000D0938900C0936B
:102A2000880015C08091B00080688093B000C0938A
:102A3000B3000DC08091B00080628093B000C0935D
:102A4000B40005C0C038D1050CF0B8CFB2CFDF91CB
:102A5000CF910895009769F0FC0101900020E9F7FB
:102A60003197AF01481B590BBC0186E594E00C94EB
:102A70009B0B80E090E008958F929F92AF92BF925F
:102A80000F931F93CF93DF93CDB7DEB7A1970FB608
:102A9000F894DEBF0FBECDBF19A2423008F44AE061
:102AA0008E010F5D1F4F842E912CA12CB12CA501FE
:102AB00094010E94BD1EE62FB901CA0101501109FF
:102AC000EA3014F4E05D01C0E95CD801EC93232BFB
:102AD000242B252B61F7C8010E942A15A1960FB659
:102AE000F894DEBF0FBECDBFDF91CF911F910F9144
:102AF000BF90AF909F908F9008950F931F93CF93A7
:102B0000DF938C01C0E0D0E0F801EC0FFD1F649171
:102B1000662371F0E0915604F09157040190F08122
:102B2000E02D86E594E00995892B11F02196ECCFF4
:102B3000CE01DF91CF911F910F910895CF93DF9335
:102B40001F92CDB7DEB7789484B5826084BD84B51A
:102B5000816084BD85B5826085BD85B5816085BD98
:102B600080916E00816080936E0010928100809150
:102B700081008260809381008091810081608093D8
:102B80008100809180008160809380008091B100FD
:102B900084608093B1008091B00081608093B00028
:102BA00080917A00846080937A0080917A008260BC
:102BB00080937A0080917A008E7F80937A00809152
:102BC0007A00806880937A001092C10061E08DE005
:102BD0000E94F41061E08DE00E94C41060E085E086
:102BE0000E94F41062E085E00E94C41061E086E07B
:102BF0000E94F41061E083E00E94F41061E084E040
:102C00000E94F41061E082E00E94F4108AE090E0FB
:102C10000E94751E8F3EC9F480E090E00E94751EF0
:102C2000809394030BE813E0EE24E394F12CC701A6
:102C30000E94751EF80181938F01FFEFEF1AFF0AC2
:102C40008AE0E816F10499F709C080919303811195
:102C5000B7C588E0809394030E94310A8091940361
:102C60000E94400A0E94BA0782E0809371048CE3BC
:102C700080937004809172048F3F09F4BDC061E0BD
:102C8000809174040E94F41061E0809176040E94A7
:102C9000F41080917604082E000C990BFC01E0578B
:102CA000F84FE491F0E0EE0FFF1FE05FFD4F25913C
:102CB000349130937D0420937C04FC01EC55F84F53
:102CC000E491E093820480917404082E000C990B27
:102CD000FC01E057F84FE491F0E0EE0FFF1FE05FDA
:102CE000FD4F2591349130937F0420937E04FC01A5
:102CF000EC55F84FE491E0938304809177048111BF
:102D00003EC061E0809172040E94F41061E0809105
:102D100073040E94F41080917304082E000C990B28
:102D2000FC01E057F84FE491F0E0EE0FFF1FE05F89
:102D3000FD4F2591349130937B0420937A04FC015C
:102D4000EC55F84FE491E093810480917204082ED1
:102D5000000C990BFC01E057F84FE491F0E0EE0F06
:102D6000FF1FE05FFD4F259134913093790420934C
:102D70007804FC01EC55F84FE491E09380048091D5
:102D80007704882309F45FC01FB7F89480919503F6
:102D9000811127C0EAE9F7E08491EEEAF7E0949127
:102DA000E82FF0E0EE0FFF1FEA5FFD4FA591B49111
:102DB000EC91E92321F461E08AE00E94C41061E013
:102DC0008AE00E94F4108CB580618CBD8CB5806463
:102DD0008CBD61E08DE00E94F41061E08BE00E9408
:102DE000F410809195038F5F809395031FBF80E55A
:102DF0008CBD81E08DBD27C01092860310928503A3
:102E000010922804109249041092260481E08093C5
:102E100025041092000461E082E10E94C41061E088
:102E200083E10E94C4108091B9008E7F8093B90025
:102E30008091B9008D7F8093B90080E28093B800C3
:102E400085E48093BC008091750487FD1EC061E01D
:102E50000E94F41061E0809175040E94C41061E04A
:102E600070E080E090E00E94301160E08091750495
:102E70000E94C4106AE070E080E090E00E9430118F
:102E800061E0809175040E94C4108EEA0E948C1348
:102E900085ED0E948C1380E80E948C1388EA0E94C2
:102EA0008C138FE10E948C1383ED0E948C1380E0C1
:102EB0000E948C1380E40E948C138DE80E948C1376
:102EC00084E10E948C1380E20E948C1380E00E94B7
:102ED0008C1381EA0E948C1388EC0E948C138AED7B
:102EE0000E948C1382E00E948C1381E80E948C1354
:102EF0008FE80E948C1389ED0E948C1381EF0E9451
:102F00008C138BED0E948C1380E40E948C1384EA56
:102F10000E948C1386EA0E948C138EE20E948C130E
:102F20008FEA0E948C130E94811380918B03882367
:102F300099F082E080936B0480915A0490915B0435
:102F400090935F0480935E0480915C0490915D0493
:102F500090936104809360040E94D5130E945714DB
:102F6000892B09F0DBC060E080E00E9440080E94ED
:102F70007B1420E000E0622F802F29830E9440080C
:102F80000E947B1429812223E9F18230D9F018F4C0
:102F9000813031F04DC4853008F04AC420E0EBCFD9
:102FA000043039F480918F03883008F041C48F5F7A
:102FB00011C00530E9F4809190038A3F08F038C4CD
:102FC0008B5F13C0043049F480918F03823008F482
:102FD0002FC4815080938F032BC4053049F4809116
:102FE0009003863008F424C485508093900320C455
:102FF000E02FF0E0E557FC4F81E09081911180E0F7
:10300000808316C4823061F018F4813021F0B3CF90
:10301000853058F0B0CF0F5F0C3009F0ACCFAACF9D
:10302000002309F403C40150A6CF0B3009F45DC09E
:103030000A3021F429830E94310A55C0093009F071
:10304000F7C313E080E290E029830E94D01468EC7B
:1030500070E080E090E00E94301180E090E00E94FB
:10306000D01468EB7BE080E090E00E9430111150BA
:1030700029811111E7CF13E080E290E029830E94BB
:10308000D01464E670E080E090E00E94301180E0AF
:1030900090E00E94D01468EE73E080E090E00E941F
:1030A0003011115029811111E7CF13E080E290E037
:1030B00029830E94D01462E370E080E090E00E94D7
:1030C000301180E090E00E94D01468EC70E080E065
:1030D00090E00E943011115029811111E7CF80E05A
:1030E00090E00E94D014298146CF0E94100A80915E
:1030F0008B03882399F082E080936B0480915A04BB
:1031000090915B0490935F0480935E0480915C04D3
:1031100090915D0490936104809360048091910389
:10312000882309F4A2C00E948113EE24E394F12CB9
:1031300000E010E02FE730E040E050E060E070E0B9
:1031400086E594E00E94EF0F81E090E0909369049F
:10315000809368049093670480936604909363045B
:103160008093620484E090E090936504809364040B
:1031700083E080936A0486E392E00E947D150BE170
:1031800010E02FE730E04BE150E060E070E086E5D2
:1031900094E00E94EF0F8FE090E09093630480939F
:1031A000620483E290E0909365048093640481E07C
:1031B00080936A0485E292E00E947D1581E290E0AE
:1031C000909363048093620482E390E0909365049B
:1031D000809364048AE192E00E947D150E94D513D9
:1031E00018EC0E945714892B09F43FC06AE070E084
:1031F00080E090E00E943011115099F7EFE17E2EAF
:10320000F0E88F2E912CA12CB12CA0E4CA2ED12C49
:10321000E12CF12C7A94772021F10E945714892B0C
:1032200021F10BEF10E001501109C1F00E94671E5F
:10323000A50194010E948B1E662E0E94671EA701A5
:1032400096010E948B1E462F50E0662D70E020E014
:1032500030E086E594E00E94C706E5CF0E94D513D2
:10326000D9CF0E9481130E94D5130E946A11DC01FC
:10327000CB01805F984DAF4FBF4F8093A6039093D3
:10328000A703A093A803B093A90379E3872E77E15E
:10329000972ECC24C394D12C6AE0A62EB12C0E9488
:1032A0007B148093AE03823009F48BC120F481300B
:1032B00009F478C1A8C1833009F4A7C0843009F0AB
:1032C000A2C1809194030E94400A3C010E94811394
:1032D000EE24E394F12C07E310E02FE730E047E31E
:1032E00050E060E070E086E594E00E94EF0FD0923D
:1032F0006904C0926804D0926704C092660481E0B9
:1033000080936A04109263041092620489E390E04F
:10331000909365048093640480919303882319F04B
:1033200084E592E002C08EE392E00E947D1560E0A9
:1033300080E00E948507230104E60E947B1481112E
:1033400041C010919303111103C083E090E002C0CB
:1033500086E090E0480E591E9AE3491697E1590617
:1033600058F0111105C03DE0432E36E1532E04C044
:1033700021EE422E24E1522EC2010E94BA0769E1D9
:1033800070E080E090E00E94301184E10E94080823
:103390008C589109B5010E94571C462FC40184190D
:1033A0009509111103C063E070E002C066E070E0AF
:1033B0000E94571C862F642FE02FE81B8E2F0E943F
:1033C0008507BBCF820104511109F4E14F0E511C56
:1033D000E12CF12CC8010E94BA0769E170E080E09D
:1033E00090E00E94301184E10E940808E816F90676
:1033F00010F438017C010E5F1F4F0415150551F7BD
:10340000C3010E94BA07C301B5C089830E9481131A
:10341000D0926904C0926804D0926704C092660496
:10342000B0926304A0926204109265041092640446
:10343000898180936A0481E892E00E947D158BE483
:1034400090E0909363048093620487E090E090930F
:1034500065048093640482E080936A048CE792E0C0
:103460000E947D15EE24E394F12C08E110E02FE793
:1034700030E048E150E060E070E086E594E00E94D2
:10348000EF0F10926304109262048BE190E090932E
:1034900065048093640481E080936A048AE692E084
:1034A0000E947D150E9410090E94D51380919403FB
:1034B0000E94400A60909303611003C023E030E053
:1034C00002C026E030E02901480E591E40FC03C02E
:1034D0008FEF481A580A82018CE3782EE12CF12CE8
:1034E000053397E1190718F40B5F1F4F07C06110F0
:1034F00003C00DE016E102C001EE14E1C8010E9414
:10350000BA0769E170E080E090E00E94301184E148
:103510000E940808E816F90610F428017C017A9444
:1035200071100AC08201045111097201E4E1EE0E2A
:10353000F11C612C712C04C08A3F910588F2F2CFF6
:10354000C8010E94BA0769E170E080E090E00E9443
:10355000301184E10E9408086816790610F42801E9
:103560003C010E5F1F4F0E151F0551F7C2010E944F
:10357000BA07C2010E94630B8093940360E070E07D
:103580000E944D0A0E946A11DC01CB014996A11DDF
:10359000B11D8093AA039093AB03A093AC03B093A7
:1035A000AD0331C0809194038F3230F0809193034A
:1035B000811105C018E01BC011E0180F18C010E001
:1035C00016C040919403403388F4242F30E080915A
:1035D0009303811103C088E090E002C080E090E096
:1035E0002817390719F01FEF140F01C01FE21093BD
:1035F0009403812F0E94400A0E94BA0760E070E0A5
:10360000812F0E944D0A8091AE03882381F00E9491
:103610006A11DC01CB01805F984DAF4FBF4F8093A3
:10362000A6039093A703A093A803B093A9030E94B5
:103630006A110091AA031091AB032091AC03309161
:10364000AD030617170728073907E0F480919203A6
:10365000882309F4B7C04090A6035090A703609058
:10366000A8037090A9030E946A11461657066806BF
:10367000790608F0A7C00E9481130E94D51381E04B
:103680008093FF03909194038091A303981781F096
:103690000E946A1100919F031091A0032091A10341
:1036A0003091A203061717072807390708F4A7C0A7
:1036B0000E946A1100919B0310919C0320919D032D
:1036C00030919E030617170728073907B8F481E0E1
:1036D00090910101911180E0809301010E946A1193
:1036E000DC01CB018C509E4FAF4FBF4F80939B03AB
:1036F00090939C03A0939D03B0939E03609101015E
:103700008DE00E94C41080918E03882309F44CC080
:10371000E0908903F0908A03E114F10409F444C0B5
:103720000E946A11009197031091980320919903C8
:1037300030919A030617170728073907C8F581E063
:1037400090919603911180E080939603882399F0DD
:10375000C60100908F0302C0880F991F0A94E2F7F8
:103760000E94D0140E946A11DC01CB018E0D9F1DB6
:10377000A11DB11D10C080E090E00E94D0140E94F5
:103780006A112091870330918803DC01CB01820FFD
:10379000931FA11DB11D8093970390939803A0934D
:1037A0009903B0939A0304C080E090E00E94D01483
:1037B00080E090E0892B09F472CD0E94000069CD71
:1037C00080E048CA84E10E9408089093A503809392
:1037D000A403BC01809194030E944D0A0E946A11C7
:1037E000DC01CB0188519C4FAF4FBF4F8093AA03A0
:1037F0009093AB03A093AC03B093AD0343CF0E946F
:10380000100A809194038093A3030E946A11DC0143
:10381000CB01805F984DAF4FBF4F80939F03909334
:10382000A003A093A103B093A20342CF0BE0A3CBCC
:1038300021E0A1CBEAE4F4E01382128288EE93E067
:10384000A0E0B0E084839583A683B7838AE193E008
:1038500091838083E6E5F4E01382128220E830E071
:103860003583248380E290E09783868331872087A5
:1038700093878287158A158614861786168681E0B7
:10388000848B2FEF3FEF338B228B318B208B868BFA
:10389000178A118E108E8AE293E0918380838FEFD6
:1038A000848F80A3868F858F84E0878F0895AA1BDD
:1038B000BB1B51E107C0AA1FBB1FA617B70710F01B
:1038C000A61BB70B881F991F5A95A9F7809590954D
:1038D000BC01CD010895EE0FFF1F0590F491E02D7E
:1038E00009940E94851C0C94661D0E945F1D58F06F
:1038F0000E94581D40F029F45F3F29F00C944F1DA1
:1039000051110C949A1D0C94551D0E94771D68F35B
:103910009923B1F3552391F3951B550BBB27AA2788
:1039200062177307840738F09F5F5F4F220F331FC2
:10393000441FAA1FA9F335D00E2E3AF0E0E832D08A
:1039400091505040E695001CCAF72BD0FE2F29D08D
:10395000660F771F881FBB1F261737074807AB075F
:10396000B0E809F0BB0B802DBF01FF2793585F4FD4
:103970003AF09E3F510578F00C944F1D0C949A1D1F
:103980005F3FE4F3983ED4F3869577956795B795B6
:10399000F7959F5FC9F7880F911D9695879597F9C1
:1039A0000895E1E0660F771F881FBB1F621773073A
:1039B0008407BA0720F0621B730B840BBA0BEE1F4F
:1039C00088F7E09508950E947F1D88F09F5798F032
:1039D000B92F9927B751B0F0E1F0660F771F881F14
:1039E000991F1AF0BA95C9F714C0B13091F00E942E
:1039F000991DB1E008950C94991D672F782F8827A1
:103A0000B85F39F0B93FCCF3869577956795B39554
:103A1000D9F73EF490958095709561957F4F8F4FC3
:103A20009F4F0895E89409C097FB3EF490958095C8
:103A3000709561957F4F8F4F9F4F9923A9F0F92F74
:103A400096E9BB279395F695879577956795B795F2
:103A5000F111F8CFFAF4BB0F11F460FF1BC06F5FD8
:103A60007F4F8F4F9F4F16C0882311F096E911C0EA
:103A7000772321F09EE8872F762F05C0662371F00B
:103A800096E8862F70E060E02AF09A95660F771F1F
:103A9000881FDAF7880F9695879597F9089597F913
:103AA0009F6780E870E060E008959FEF80EC0895E4
:103AB00000240A941616170618060906089500240D
:103AC0000A9412161306140605060895092E039487
:103AD000000C11F4882352F0BB0F40F4BF2B11F4FB
:103AE00060FF04C06F5F7F4F8F4F9F4F089557FD5A
:103AF0009058440F551F59F05F3F71F04795880F5C
:103B000097FB991F61F09F3F79F0879508951216F2
:103B100013061406551FF2CF4695F1DF08C016169E
:103B200017061806991FF1CF86957105610508944F
:103B30000895E894BB2766277727CB0197F9089566
:103B40000E94B31D0C94661D0E94581D38F00E94FF
:103B50005F1D20F0952311F00C944F1D0C94551D02
:103B600011240C949A1D0E94771D70F3959FC1F348
:103B7000950F50E0551F629FF001729FBB27F00D1B
:103B8000B11D639FAA27F00DB11DAA1F649F662770
:103B9000B00DA11D661F829F2227B00DA11D621FBF
:103BA000739FB00DA11D621F839FA00D611D221F79
:103BB000749F3327A00D611D231F849F600D211D5D
:103BC000822F762F6A2F11249F5750409AF0F1F0E0
:103BD00088234AF0EE0FFF1FBB1F661F771F881F49
:103BE00091505040A9F79E3F510580F00C944F1D15
:103BF0000C949A1D5F3FE4F3983ED4F38695779535
:103C00006795B795F795E7959F5FC1F7FE2B880FEE
:103C1000911D9695879597F9089581E090E0F89425
:103C20000C94EE1EFB01DC0101900D920020E1F7E7
:103C300008958F929F92AF92BF92CF92DF92EF92B0
:103C4000FF92CF93DF93EC01688179818A819B8118
:103C5000611571058105910521F464E279ED8BE52B
:103C600097E02DE133EF41E050E00E948B1E4901C7
:103C70005A019B01AC01A7EAB1E40E94AA1E6B01A4
:103C80007C01ACEEB4EFA50194010E94B81EDC01EA
:103C9000CB018C0D9D1DAE1DBF1DB7FF03C001974D
:103CA000A109B04888839983AA83BB83BC01CD0155
:103CB0009F77DF91CF91FF90EF90DF90CF90BF90F3
:103CC000AF909F908F9008950E94191E089582E0F2
:103CD00093E00E94191E08956093020370930303FA
:103CE00080930403909305030895F999FECF92BD44
:103CF00081BDF89A992780B50895262FF999FECFAE
:103D00001FBA92BD81BD20BD0FB6F894FA9AF99AF8
:103D10000FBE01960895052E97FB1EF400940E9495
:103D2000A21E57FD07D00E94BD1E07FC03D04EF413
:103D30000C94A21E50954095309521953F4F4F4FC2
:103D40005F4F089590958095709561957F4F8F4F47
:103D50009F4F08950E94DF1EA59F900DB49F900D68
:103D6000A49F800D911D11240895B7FF0C94AA1EE5
:103D70000E94AA1E821B930B0895A1E21A2EAA1B71
:103D8000BB1BFD010DC0AA1FBB1FEE1FFF1FA2170B
:103D9000B307E407F50720F0A21BB30BE40BF50B08
:103DA000661F771F881F991F1A9469F76095709591
:103DB000809590959B01AC01BD01CF010895A29F14
:103DC000B001B39FC001A39F700D811D1124911DEF
:103DD000B29F700D811D1124911D0895F894FFCF9D
:103DE0000E010000000000000000000000000000C4
:103DF00000000000000000000000000000000000C3
:103E000000000000000000000000000000000000B2
:103E100000000000000000000000000000000000A2
:103E20000080808000000000000000000000000012
:103E30000000008080C0C000000000000000000002
:103E40000000000000000000000000000000000072
:103E50000000000000000000000000000000000062
:103E60000000000000000000000000000000000052
:103E700000000000000080C0E0F0F8FCF8E0000066
